:100000000C94AC070C94F0070C94F0070C94F007D8
:100010000C94F0070C94F0070C94F0070C94F00784
:100020000C94F0070C94F0070C9415130C94E71340
:100030000C94F0070C94F0070C94F0070C94F00764
:100040000C94F0070C94BF2C0C94F0070C94F00760
:100050000C94F0070C94C6220C94F0070C94F00753
:100060000C94F0070C94F0070C94F0070C94F00734
:100070000C94F0070C94F0070C94F0070C94F00724
:100080000C94F0070C94F0070C94F0070C94F00714
:100090000C94F0070C94F0070C94F0070C94F00704
:1000A0000C94F0070C94F0070C94F0074C146E14A9
:1000B00059156E145915B014D314591528153B153C
:1000C00089188918B718B718FA183619371B371B4B
:1000D0004E19371B451A451A111B371B371B251B99
:1000E0000000F0A1F0A329002B000354E1003581AA
:1000F00000001E00140004001D7164004D001F006C
:100100001A0016001B00E1044C0020000800070044
:10011000060050002A0021001500090019004F00B8
:100120004A00220017000A000500000002541908C6
:10013000E3000000E20000002E770608E700000060
:10014000E60000002E7F23001C000B0011000000C1
:100150000454240018000D00100052004B0025002C
:100160000C000E00360051002C00260012000F007B
:100170003700E108280027001300330038713000F1
:100180004E002D002F003482E50031810000010077
:10019000010001000100010000003A0035003100BB
:1001A0000100010001003B00350221026400010052
:1001B0004C003C001E0224062202010001003D000A
:1001C0002D0224022404010001003E00010037003A
:1001D0001104000001000100010000000100000006
:1001E00001000100010000000100000001003F00CB
:1001F00024062402230200000100400022042502FC
:1002000035000100010041002304260235023700B9
:1002100001004200240425041F021E0201004300C5
:1002200031002604310201000100440045000100B4
:100230002D02010000000100010001000100010089
:100240000000010001000100FB00010001000100AD
:100250000100F200F900010001000100F000F100CE
:10026000FA00F400010001000100F300FC00F500B9
:100270000100010001000100F60000000100010082
:100280000100000001000000010001000100000069
:100290000100000001000100010001000100000058
:1002A0000100010001000100A800A90001000100F7
:1002B00001000100AC00AA00B6000100010001002D
:1002C000AB0050000100010001000100520051008C
:1002D0000100AE000100010001004F00000001001C
:1002E0000100010001000100000001000E000B00F0
:1002F0001B7101000100010037000400140001001F
:10030000010001001200080034000100010001009A
:1003100036000C002F000100010001001D00180034
:100320003300000001000100010000000100000096
:1003300001000100010000000100000001000100B7
:100340001900070005000000010001000A00170065
:100350001300010001000100060015001A00010051
:10036000010001000F001100100001000100010058
:100370002D0016000D710100010038001C000982DB
:100380000100010000000100010001000100010066
:100390000000010001000100010001000100010056
:1003A0000100500001000100010001005200510055
:1003B000010001000100010001004F0001000100E7
:1003C0000100010001000100010000000100010026
:1003D0000100000001000000010001000100000018
:1003E0000100000001003F00520051002302000004
:1003F00001004000240021001E00270001004100F0
:10040000250022001F0037000100420026002300C3
:1004100020002700010043003002300024022E009B
:1004200001004400450001000100010000000A0035
:100430002530313662003A200025303258000A72E9
:100440002F63203031323334353637383941424327
:100450004445460A000A002530325800626F756E26
:100460006365213A20006C656674207369646520B9
:1004700061747461636865640A006C6566742073F6
:10048000696465206E6F7420726573706F6E646945
:100490006E670A00747279696E6720746F207265E6
:1004A000736574206D637032333031380A000A444A
:1004B000454255473A20656E61626C65642E0A00BC
:1004C0005B735D004B6579626F6172642073746168
:1004D00072742E0A005B575D005B535D005B525DDA
:1004E000005B445D005B435D0016034500720067DE
:1004F000006F0044006F007800200045005A0000A3
:100500000016034500720067006F0044006F00781A
:1005100000200045005A0000000403090409028D70
:1005200000050100A0FA090400000103010100090F
:100530002111010001223F000705810308000A097B
:100540000401000103010200092111010001224DF3
:10055000000705820308000A0904020001030000E5
:10056000000921110100012236000705830308005C
:100570000A0904030002030000000921110100011F
:100580002220000705840320000107050403200042
:100590000109040400010300000009211101000108
:1005A0002239000705850310000112011001000027
:1005B0000008EDFE07130100010200010501090614
:1005C000A101050719E029E7150025019508750126
:1005D000810205081901290595057501910295010A
:1005E00075039101050719002977150025019578F4
:1005F00075018102C00631FF0974A101097515005A
:1006000025FF9520750881020976150025FF9520A4
:1006100075089102C005010980A10185021601003B
:1006200026B7001A01002AB700751095018100C095
:10063000050C0901A1018503160100269C021A017F
:10064000002A9C02751095018100C005010902A1D4
:10065000010901A1000509190129051500250195C8
:1006600005750181029501750381010501093009B4
:10067000311581257F950275088106093815812578
:100680007F950175088106050C0A38021581257FC2
:10069000950175088106C0C005010906A10105077D
:1006A00019E029E7150025019508750181029501DA
:1006B0007508810105081901290595057501910243
:1006C0009501750391010507190029FF150025FF04
:1006D000950675088100C00A002530325820006B4D
:1006E0006579626F6172645F7265706F72743A20CF
:1006F000000A0025303258006B6579626F617264C0
:100700005F7365745F6C65643A200064656C5F6B51
:1007100065795F6269743A2063616E27742064654D
:100720006C3A20253032580A006164645F6B657949
:100730005F6269743A2063616E2774206164643A71
:1007400020253032580A00646F6E652E0A00626FF1
:100750006F676D61676963207363616E3A202E2E47
:100760002E2000290A002575002F002575005D2820
:10077000002564002000256400200025640020007E
:100780002564007C0025303258006D6F7573656BF1
:100790006579205B62746E7C782079207620685DB4
:1007A000287265702F61636C293A205B006D6B5F66
:1007B000776865656C5F74696D655F746F5F6D61A7
:1007C00078203D2025640A006D6B5F776865656C55
:1007D0005F6D61785F7370656564203D2025640AF4
:1007E000006D6B5F74696D655F746F5F6D6178201C
:1007F0003D2025640A006D6B5F6D61785F737065E5
:100800006564203D2025640A006D6B5F696E746528
:100810007276616C203D2025640A006D6B5F646513
:100820006C6179203D2025640A006D6B5F776865F7
:10083000656C5F74696D655F746F5F6D6178203D95
:100840002025640A006D6B5F776865656C5F6D617C
:10085000785F7370656564203D2025640A006D6BC8
:100860005F74696D655F746F5F6D6178203D2025F1
:10087000640A006D6B5F6D61785F737065656420FD
:100880003D2025640A006D6B5F696E746572766148
:100890006C203D2025640A006D6B5F64656C617996
:1008A000203D2025640A000A00257500363A20778D
:1008B0006865656C5F74696D655F746F5F6D6178A5
:1008C0003A20000A00257500353A20776865656C86
:1008D0005F6D61785F73706565643A20000A00257A
:1008E0007500343A2074696D655F746F5F6D61786F
:1008F0003A20000A00257500333A206D61785F7355
:10090000706565643A20000A00257500323A206956
:100910006E74657276616C286D73293A20000A0046
:10092000257500313A2064656C6179282A31306D73
:1009300073293A20000A092D2056616C75657320D1
:100940002D0A004D3E004D25643E20003F0073659A
:10095000742064656661756C740A00433E200077FC
:10096000686572652064656C74613A2063757273A2
:100970006F723D25642C20776865656C3D25640A9F
:1009800053656520687474703A2F2F656E2E7769F1
:100990006B6970656469612E6F72672F77696B6927
:1009A0002F4D6F7573655F6B6579730A000A092DAA
:1009B000204D6F7573656B6579202D0A4553432F64
:1009C000713A09717569740A313A0964656C617923
:1009D000282A31306D73290A323A09696E746572BA
:1009E00076616C286D73290A333A096D61785F73FB
:1009F000706565640A343A0974696D655F746F5F88
:100A00006D61780A353A09776865656C5F6D617864
:100A10005F73706565640A363A09776865656C5F6F
:100A200074696D655F746F5F6D61780A0A703A0969
:100A30007072696E742076616C7565730A643A0928
:100A40007365742064656661756C74730A75703AB9
:100A5000092B310A646F776E3A092D310A70677578
:100A6000703A092B31300A7067646F776E3A092D3E
:100A700031300A0A7370656564203D2064656C74CA
:100A800061202A206D61785F7370656564202A207B
:100A900028726570656174202F2074696D655F74BC
:100AA0006F5F6D6178290A003F004D3E2000433E94
:100AB00020004C25640A000A092D20436F6E736FD5
:100AC0006C65202D0A4553432F713A09717569747D
:100AD0000A6D3A096D6F7573656B65790A000A09CD
:100AE0002D204D61676963202D0A643A09646562AF
:100AF00075670A783A096465627567206D6174727A
:100B000069780A6B3A096465627567206B6579627A
:100B10006F6172640A6D3A096465627567206D6F72
:100B20007573650A763A0976657273696F6E0A7332
:100B30003A097374617475730A633A09636F6E736B
:100B40006F6C65206D6F64650A302D343A096C61F5
:100B5000796572302D34284631302D4634290A50BB
:100B60006175733A09626F6F746C6F616465720AC4
:100B7000653A09656570726F6D0A6E3A094E4B529F
:100B80004F0A7A3A09736C656570204C45442074AD
:100B90006573740A000A002575002E6E6B726F3A39
:100BA00020000A002575002E737761705F62616313
:100BB0006B736C6173685F6261636B7370616365B3
:100BC0003A20000A002575002E737761705F677206
:100BD0006176655F6573633A20000A002575002E13
:100BE0006E6F5F6775693A20000A002575002E73E5
:100BF0007761705F72616C745F726775693A20002B
:100C00000A002575002E737761705F6C616C745FEC
:100C10006C6775693A20000A002575002E636170C3
:100C2000736C6F636B5F746F5F636F6E74726F6C06
:100C30003A20000A002575002E737761705F636F9C
:100C40006E74726F6C5F636170736C6F636B3A206C
:100C5000000A0025303258006B65796D61705F6362
:100C60006F6E6669672E7261773A20000A002575FB
:100C7000002E6D6F7573653A20000A002575002EF1
:100C80006B6579626F6172643A20000A0025750015
:100C90002E6D61747269783A20000A002575002E65
:100CA000656E61626C653A20000A0025303258009A
:100CB00064656275675F636F6E6669672E726177E0
:100CC0003A20000A0025750064656661756C745FE2
:100CD0006C617965723A20003F004E4B524F3A20CA
:100CE0006F66660A004E4B524F3A206F6E0A0074D0
:100CF000696D65725F636F756E743A202530346C70
:100D0000580A006B6579626F6172645F6E6B726F17
:100D10003A2025580A006B6579626F6172645F69D9
:100D2000646C653A2025580A006B6579626F6172C0
:100D3000645F70726F746F636F6C3A2025580A009D
:100D4000686F73745F6B6579626F6172645F6C6505
:100D5000647328293A2025580A000A092D20537463
:100D600061747573202D0A004743433A20342E38AE
:100D70002E32204156522D4C4942433A20312E38D2
:100D80002E30204156525F415243483A20617672DC
:100D9000350A004F5054494F4E533A204C55464166
:100DA00020424F4F544D41474943204D4F555345E5
:100DB0004B45592045585452414B455920434F4EBD
:100DC000534F4C4520434F4D4D414E44204E4B52C6
:100DD0004F203531320A004255494C443A2037669B
:100DE00038346162362D6469727479202830333A60
:100DF00032393A3336204A616E2032322032303175
:100E000036290A005649443A203078464545442858
:100E10004572676F446F7820455A29205049443AFB
:100E200020307831333037284572676F446F78202F
:100E3000455A29205645523A203078303030310A10
:100E400000444553433A20742E6D2E6B2E206B6563
:100E500079626F617264206669726D776172652074
:100E6000666F72204572676F646F780A000A092DF9
:100E70002056657273696F6E202D0A000A6D6F75BA
:100E800073653A206F66660A000A6D6F7573653A7E
:100E9000206F6E0A000A6B6579626F6172643A2096
:100EA0006F66660A000A6B6579626F6172643A2048
:100EB0006F6E0A000A6D61747269783A206F666617
:100EC0000A000A6D61747269783A206F6E0A000A2E
:100ED00064656275673A206F6E0A000A6465627520
:100EE000673A206F66660A000A0A626F6F746C6F59
:100EF000616465722E2E2E2000433E2000656563DE
:100F00006F6E6669673A0A00536C656570204C45E0
:100F10004420746573740A000000000000000000A3
:100F2000000000010204060A0F17202C3A4A5D71E6
:100F3000879DB3C7DAE9F5FCFFFCF5E9DAC7B39D95
:100F400087715D4A3A2C20170F0A0604020100003F
:100F5000000000000000000011241FBECFEFDAE007
:100F6000DEBFCDBF04B603FE24C08091F90190918D
:100F7000FA01A091FB01B091FC018730904BA74092
:100F8000B04BB9F41092F9011092FA011092FB01E2
:100F90001092FC0114BE84B7877F84BF88E10FB62E
:100FA000F89480936000109260000FBEE0E0FFE3D1
:100FB000099511E0A0E0B1E0EAE1FDE502C005908D
:100FC0000D92AA33B107D9F711E0AAE3B1E001C04D
:100FD0001D92A93FB107E1F70E944F100C948B2E90
:100FE0000C940000FF93EF93E0913A01F0913B01E4
:100FF000309709F00995EF91FF910895FC018591D3
:10100000803011F0EFDFFBCF0895FF27E0E230E200
:1010100047FF0CC0419597FF09C0EDE260957095C0
:1010200080959095611D711D811D911D27FF02C046
:10103000219530E350E2AA27660F771F881F991F7A
:10104000AA1FA41710F0A41B63955A95A9F7AA30FC
:1010500008F0A95FA05DAF93F39561157105810557
:10106000910541F7ED3211F4EF93F395F21718F46F
:101070003F93F395FBCF8F91B5DFFA95E1F7089594
:10108000E991F9918591803021F0853219F0AADF3C
:10109000F9CF089520E0E89455915532C1F35033CB
:1010A00011F4689455915A3348F4505390F3220F39
:1010B000022E220F220F200D250FF4CF0EF42195C2
:1010C00089919991533619F3533729F1533559F1D1
:1010D000BC0188279927E8945C3621F4899199917D
:1010E00068945591543639F446EF7EF077FF0DC081
:1010F0008FEF9FEF0AC055374AE039F0583540E18D
:1011000021F0523642E009F00895FF93EF937DDF1E
:10111000EF91FF91B7CFFF93EF93FC018191803066
:10112000B9F360DFFBCFFF93EF9368DFF1CFDF937D
:10113000CF93CDB7DEB72596A3DFCF91DF9108958A
:1011400061110BC0FC018281882321F085EE0E9491
:101150001D1703C085EE0E94E51780E090E008951A
:1011600008956091BC017091BD018091BE01909184
:10117000BF010E94CA2156985E9825982D982698FE
:101180002E9827982F98823061F018F4813031F032
:101190000895833049F0843051F00895259A2D9AAE
:1011A0000895269A2E9A0895279A2F9A0895259A97
:1011B0002D9A279A2F9A089581EB98E0892B11F0A8
:1011C0000E94B10880E090E0089556985E982598B6
:1011D0002D9826982E9827982F988FEF90E090932F
:1011E00089008093880090938B0080938A0090936D
:1011F0008D0080938C00259A2D9A2FEF80E792E046
:10120000215080409040E1F700C00000269A2E9ABD
:101210002FEF80E792E0215080409040E1F700C03E
:101220000000279A2F9A2FEF80E792E0215080400C
:101230009040E1F700C0000025982D982FEF80E73F
:1012400092E0215080409040E1F700C000002698D5
:101250002E982FEF80E792E0215080409040E1F7F8
:1012600000C0000027982F9856985E9825982D98D2
:1012700026982E9827982F98089589EA80938000C1
:1012800089E08093810024982C983F988AB18F74CC
:101290008AB96E98479A8BB1806B8BB9769A0E9407
:1012A000E50880EB98E0892B11F00E94B00880E0FF
:1012B00090E0089580E28093000180913C018111CB
:1012C0000EC00E94A90981E080933C012FEF83EDBD
:1012D00090E3215080409040E1F700C0000080E49E
:1012E0000E94AF098093000181112EC00E94D9098C
:1012F00080930001811128C00E94D90980930001C8
:10130000811122C08FE30E94D909809300018111CD
:101310001BC00E94D10980E40E94AF0980930001A4
:10132000811112C08CE00E94D909809300018111C3
:101330000BC00E94D90980930001811105C08FE381
:101340000E94D909809300010E94D1098091000177
:1013500008951092B9008AE08093B800089594EA45
:101360009093BC009091BC0097FFFCCF9091B90086
:10137000987F983021F0903111F081E008958093AA
:10138000BB0084E88093BC008091BC0087FFFCCF49
:101390008091B900887F883111F0803471F780E046
:1013A000089584E98093BC008091BC0084FDFCCF4B
:1013B00008958093BB0084E88093BC008091BC00BA
:1013C00087FFFCCF9091B900987F81E0983209F4B3
:1013D00080E0089584E88093BC008091BC0087FF82
:1013E000FCCF8091BB00089580910001811115C050
:1013F00080E40E94AF098093000181110CC082E15A
:101400000E94D90980930001811105C08FEF0E94CD
:10141000D909809300010E94D10984B1807F84B9E9
:1014200085B1807F85B98AB1837F8AB98BB1837F8B
:101430008BB93E98469808950E945A0980930001FE
:101440000E94F40980B38C7080BB81B3836F81BB31
:10145000ECE4F1E0AEE3B1E011921D9281E0EA35F7
:10146000F807D1F78DE399E0892B11F00C943D0931
:1014700008959F92AF92BF92CF92DF92EF92FF9228
:101480000F931F93CF93DF93809100018823E1F0A6
:1014900080913D018F5F80933D01811115C084E9EA
:1014A00094E00E94FE070E945A098093000188235D
:1014B00029F08AE794E00E94FE0706C086E694E0E1
:1014C0000E94FE070E94E5080EE311E0C0E0D0E0B4
:1014D000BB24B39482E0A82ECC24C394D12C27E55E
:1014E000E22E24E0F22EC73000F580910001811138
:1014F00062C080E40E94AF0980930001811112C094
:1015000082E10E94D9098093000181110BC0C601BC
:101510000C2E01C0880F0A94EAF780950E94D90921
:10152000809300010E94D10946C0CA30A1F028F47E
:10153000C83059F0C93061F005C0CC3089F070F086
:10154000CD3089F0209A289810C0219A29980DC092
:10155000229A2A980AC0239A2B9807C0529A01C04F
:10156000539A5B9802C03E9A4698E0EAEA95F1F7F2
:101570008FB1799985C092E081708B25892B7C9BF6
:1015800002C090E001C094E0892B7D9B02C090E0F6
:1015900001C098E0892B7E9B02C090E001C090E1E1
:1015A000892B9FB19095991F9927991F9295990F13
:1015B000907E892B10C080910001811176C080E45B
:1015C0000E94AF0980930001882309F45BC0912C2D
:1015D0000E94D109892DF8019081981739F18083F3
:1015E00080910101882301F18091D70180FF04C01F
:1015F0008CE594E00E94FE078091D70180FF0CC02B
:10160000809101011F928F93FF92EF920E949708A1
:101610000F900F900F900F908091D70180FF04C022
:1016200085E594E00E94FE07A09201010E94F40962
:1016300021960F5F1F4FCE30D10509F054CF809116
:1016400001018823B1F0815080930101882339F092
:101650008FE99FE00197F1F700C000000AC0ACE4F9
:10166000B1E0EEE3F1E081918D9391E0EC34F90784
:10167000D1F78CED98E0892BD1F00E94DC0817C0DF
:1016800090E07ACF83E10E94D90980930001811113
:101690009ECF81E40E94AF0980930001811197CF12
:1016A0000E94EA09982E909493CF80E094CF81E035
:1016B000DF91CF911F910F91FF90EF90DF90CF902E
:1016C000BF90AF909F900895E82FF0E0E45BFE4F4D
:1016D00080810895CF92DF92EF92FF920F931F9334
:1016E000CF93DF938EE394E00E94FE073CE4E32E69
:1016F00031E0F32EC0E0D0E049E3C42E44E0D42E24
:1017000000E314E0DF93CF93DF92CF920E9497081B
:1017100086E394E00E94FE07F70181917F0190E04B
:101720000E942F229F938F931F930F930E949708DD
:101730008EE294E00E94FE0721968DB79EB7089630
:101740000FB6F8949EBF0FBE8DBFCE30D105D1F637
:10175000DF91CF911F910F91FF90EF90DF90CF908D
:1017600008958B3B910578F4883A910540F5853AC8
:101770009105D0F48430910508F0B1C08130910515
:1017800009F4ADC06BC0803E910508F467C0883E87
:10179000910508F4A4C09C01205F31092031310576
:1017A00008F05CC090650895853A910509F459C028
:1017B000863A910509F458C083E890E40895883A80
:1017C000910509F454C0893A910509F453C08A3A45
:1017D000910509F452C08B3A910509F451C08C3A35
:1017E000910509F450C08D3A910509F44FC0803B32
:1017F000910509F44EC08E3A910509F44DC08F3A17
:10180000910509F44CC0813B910509F44BC0823B22
:10181000910509F44AC0833B910509F449C0843B12
:10182000910509F448C0853B910509F447C0863B02
:10183000910509F446C0873B910509F445C0883BF2
:10184000910509F444C0893B910509F443C08A3BE2
:10185000910509F042C08AE296E4089580E090E0A4
:10186000089581E890E4089582E890E4089582EE76
:1018700094E4089589EE94E408958AEE94E408953A
:1018800085EB94E4089586EB94E4089587EB94E463
:1018900008958CEC94E408958DEC94E4089583E825
:1018A00095E408958AE895E4089582E995E4089519
:1018B00084E995E4089581E296E4089583E296E44C
:1018C000089584E296E4089585E296E4089586E218
:1018D00096E4089587E296E4089580E094E40895FC
:1018E000089596E0799FF001112494E5899FE00D19
:1018F000F11D1124E60FF11DEE0FFF1FEA51FF4FFE
:10190000859194910895880F991F805A9040FC0109
:10191000859194910895880F991F80529F4FFC01E3
:1019200085919491089526E0729FF001112444E579
:10193000849FE00DF11D1124E60FF11DEE0FFF1F36
:10194000EA51FF4F25913491C9019A9581159F4124
:1019500010F4C9010895C90190528115904128F4ED
:10196000C9019F700E948B0C0895C9019053811585
:10197000904120F4C9019927906C0895211580E5C4
:10198000380769F40E94581B9FEF24E34CE0915004
:1019900020404040E1F700C000000C94EB222130D1
:1019A00080E5380751F48EEA94E00E94FE078091AA
:1019B000D70181608093D7010895C90190558115A1
:1019C000904108F050C0832F99278F70992781305C
:1019D0009105D9F4A9014370552702C0880F991FBA
:1019E0004A95E2F79C68A90164E0440F551F6A9587
:1019F000E1F744275370842B952B73E0220F331F9C
:101A00007A95E1F7207633271DC08230910529F4BD
:101A1000922F8827816F906A089583309105A9F4E9
:101A2000A9014370552781E090E002C0880F991FFB
:101A30004A95E2F79C6843E0220F331F4A95E1F78D
:101A4000207E3770822B932B08950497F1F4A9011F
:101A50004370552781E090E002C0880F991F4A9596
:101A6000E2F79A68E8CFC90190578115904120F4B8
:101A7000C9019F7090620895C901905881159041E5
:101A800020F4C9019F70906A0895203E3105E0F46A
:101A9000203C310558F52133310509F470C048F474
:101AA0002932310509F464C02A32310509F46EC0C7
:101AB00074C029333105F1F022383105D9F02533CE
:101AC000310509F44EC069C0233E310589F138F46F
:101AD000203E3105C1F0223E3105E1F05EC0263ED8
:101AE000310569F1273E3105A9F157C0C9010E94AE
:101AF000830C08958091EA0180FD02C081FF4DC0F2
:101B000080EE90E04BC08091EA0180FFF9CF89E33D
:101B100090E044C08091EA0182FF0EC08091EA010A
:101B200084FF03C080E090E039C083EE90E036C0CF
:101B30008091EA0182FFF2CF82EE90E02FC0809187
:101B4000EA0183FF0BC08091EA0184FDEBCF87EEB1
:101B500090E024C08091EA0183FFF5CF86EE90E00B
:101B60001DC08091EA0185FF07C089E290E016C0A0
:101B70008091EA0185FFF9CF85E390E00FC0809165
:101B8000EA0186FF07C08AE290E008C08091EA017E
:101B900086FFF9CF81E390E001C0C9010E94B10B3B
:101BA0000895089580916D0108959FB7F89410925B
:101BB0005C019FBF9091F001943009F058C0909162
:101BC000E9009F702091EC0020FF02C020E801C0D6
:101BD00020E0292B94E09093E9009091EB0090FF96
:101BE00043C09091EE0097FF3FC090915A01992316
:101BF00021F09091E80095FF37C010925A0196E0CD
:101C00003091E80035FD15C03091F001343061F5B8
:101C10003091EB0035FD28C0915021F481E0809394
:101C20005A0122C0EFE9FFE03197F1F700C0000050
:101C3000E7CF8093F1008091E80085FD0AC0809194
:101C4000E80080FFFCCF8091E8008E778093E80069
:101C500006C08FB7F89491E090935C018FBF2F700E
:101C60002093E90080E008952F702093E9008FEF22
:101C70000895CF93DF9300D01F92CDB7DEB72091A8
:101C8000F001243019F523E029839B838A83209374
:101C9000E9008FEF9091E800815095FD06C095ED29
:101CA0009A95F1F700008111F5CF8091E80085FF4A
:101CB0000DC040E050E063E070E0CE0101960E946C
:101CC00008118091E8008E778093E8000F900F90C4
:101CD0000F90DF91CF910895CF93DF9300D01F92A3
:101CE000CDB7DEB72091F001243021F522E0298321
:101CF0009B838A8383E08093E9008FEF9091E800D3
:101D0000815095FD06C095ED9A95F1F7000081117F
:101D1000F5CF8091E80085FF0DC040E050E063E022
:101D200070E0CE0101960E9408118091E8008E7744
:101D30008093E8000F900F900F90DF91CF9108955E
:101D40002091F0012430F1F422E02093E9002FEFFC
:101D50003091E800215035FD06C035ED3A95F1F798
:101D600000002111F5CF2091E80025FF0BC040E0D5
:101D700050E065E070E00E9408118091E8008E77E5
:101D80008093E8000895CF93DF93EC018091F001F8
:101D9000843009F047C080910C018823E1F08091E4
:101DA0000D018823C1F085E08093E9008FEF9091C9
:101DB000E800815095FD06C095E19A95F1F7000085
:101DC0008111F5CF8091E80085FF2CC040E050E004
:101DD00060E170E017C081E08093E9008FEF90919F
:101DE000E800815095FD06C095ED9A95F1F7000049
:101DF0008111F5CF8091E80085FF14C040E050E0EC
:101E000068E070E0CE010E9408118091E8008E77B2
:101E10008093E80080E1FE01ADE5B1E001900D9214
:101E20008A95E1F7DF91CF91089585EE94E00E94C5
:101E3000FE078091EF01811109C00E949A120E9451
:101E4000F7128091E20084608093E200089581EEB1
:101E500094E00E94FE071092EF0108958DED94E04A
:101E60000C94FE0789ED94E00E94FE070C94AC2CC4
:101E700085ED94E00E94FE070E9486220E94B22C0B
:101E80000E9493150C94D10D80915B018F5F80931C
:101E90005B0162E30E94202E911135C010925B011C
:101EA00080915C01882379F18091F001843049F5BB
:101EB0008091E9008F709091EC0090FF02C090E853
:101EC00001C090E0982B84E08093E9008091EB00C2
:101ED00080FF14C08091EE0087FF10C08091E80061
:101EE00085FF03C01092F100F9CF8091E80080FFD8
:101EF00005C08091E8008E778093E8009F709093F2
:101F0000E90010925C01089542E061EC81E00E94DA
:101F1000141242E061EC82E00E94141242E061EC93
:101F200083E00E94141242E261EC84E00E941412E9
:101F300042E161EC85E00C9414128091F20183304F
:101F400009F455C030F4813071F0823009F48EC04C
:101F500008958A3009F47AC08B3009F460C0893062
:101F600009F09CC020C08091F101813A09F096C02F
:101F70008091E800877F8093E8008091F50190913F
:101F8000F601892B21F060E080E090E003C060E181
:101F90008DE591E070E00E9451118091E8008B770F
:101FA0008093E80008958091F101813209F076C0B4
:101FB0008091F5019091F601009719F0049709F0CE
:101FC0006DC08091E800877F8093E8008091E800F1
:101FD00082FD05C08091F0018111F8CF5FC0809132
:101FE000F10080936D018091E8008B7753C0809160
:101FF000F101813A09F052C08091F5019091F6010A
:10200000892B09F04BC08091E800877F8093E8001E
:102010008091E80080FFFCCF80910C0136C0809158
:10202000F1018132D9F58091F5019091F601892B6A
:10203000A9F58091E800877F8093E8000E9449120B
:102040008091F30180930C010C94581B8091F10155
:10205000813221F58091E800877F8093E8000E941B
:1020600049128091F40180936E0108958091F101ED
:10207000813AA1F48091E800877F8093E800809105
:10208000E80080FFFCCF80916E018093F100809189
:10209000E8008E778093E8000C944912089584B785
:1020A000877F84BF88E10FB6F89480936000109218
:1020B00060000FBE90E080E80FB6F8948093610056
:1020C000909361000FBE0E941C160E949A120E94FB
:1020D000F7128091E20084608093E20085ED9DE03C
:1020E0000E94C52178940E9471150E941E1682E0FC
:1020F00091E00E948E150E949A2C84EC94E00E943C
:10210000FE078091F001853089F480EC94E00E9414
:10211000FE070E9449228091EE01882391F30E94DC
:102120007122882371F30E94F210EBCF0E944C16AB
:10213000E8CF292F332723303105A9F06CF4213063
:10214000310509F442C02230310509F043C08DE861
:1021500090E02DE135E042C021323105C9F0223254
:10216000310519F137C099278130910541F082304E
:10217000910541F0892B71F5E9E1F5E005C0E1E059
:10218000F5E002C0E9EEF4E0849190E09F0126C002
:10219000653000F5E62FF0E0EE0FFF1FEB5DFE4F20
:1021A0002081318189E090E019C0653098F4E62FF4
:1021B000F0E0DF01AA0FBB1FA55EBE4F2D913C9141
:1021C000EA5EFE4F808190E009C082E190E02AEA59
:1021D00035E004C080E090E020E030E0FA01318397
:1021E0002083089580E189BD82E189BD09B400FEA4
:1021F000FDCF8091D8008F7D8093D8008091E00042
:1022000082608093E0008091E00081FDFCCF089522
:10221000CF92DF92EF92FF920F931F93CF93DF93B2
:102220007C018B01EA010E946A12811131C0209762
:1022300031F088819981081B190BE80EF91EC12C19
:10224000D12C0115110519F18091E80085FD14C00C
:102250008091E8008E778093E800209741F0888194
:1022600099818C0D9D1D9983888385E011C00E9402
:102270006A12882331F30CC0F70181917F018093AA
:10228000F10001501109FFEFCF1ADF0ADACF80E029
:10229000DF91CF911F910F91FF90EF90DF90CF9042
:1022A00008952091F7013091F8012617370748F07B
:1022B0006115710539F42091E8002E772093E8002C
:1022C00001C0B901FC0120E061157105B9F18091EF
:1022D000F001882309F440C0853009F43FC08091A3
:1022E000E80083FD3DC08091E80082FF06C0809138
:1022F000E80082FF26C080E008958091E80080FF1A
:10230000E3CF2091F3008091F20090E0922B6115D1
:10231000710551F08830910538F421912093F10036
:10232000615071090196F3CF21E0089709F020E090
:102330008091E8008E778093E800C6CF2111C7CF47
:10234000D6CF8091F001882339F0853039F0809123
:10235000E80083FFCCCF04C082E0089583E00895B5
:1023600081E008952091F7013091F8012617370791
:1023700048F06115710539F42091E8002E7720931B
:10238000E80001C0B901FC0120E061157105C1F14F
:102390008091F001882309F441C0853009F440C0E0
:1023A0008091E80083FD3EC08091E80082FF06C076
:1023B0008091E80082FF27C080E008958091E800C6
:1023C00080FFE3CF2091F3008091F20090E0922B08
:1023D0006115710559F08830910540F424912093DE
:1023E000F1003196615071090196F2CF21E0089712
:1023F00009F020E08091E8008E778093E800C5CF57
:102400002111C6CFD5CF8091F001882339F08530D6
:1024100039F08091E80083FFCBCF04C082E00895BB
:1024200083E0089581E00895982F973058F59093B0
:10243000E900981739F07091EC002091ED0050916F
:10244000F00003C0242F762F50E021FF19C03091F7
:10245000EB003E7F3093EB003091ED003D7F3093F9
:10246000ED003091EB0031603093EB007093EC00A5
:102470002093ED005093F0002091EE0027FF07C05D
:102480009F5FD3CF8F708093E90081E0089580E053
:1024900008958091F10187FD05C08091E80080FFDB
:1024A0000EC012C08091E80082FD05C08091F0014D
:1024B0008111F8CF08958091E8008B7708C0809152
:1024C000F0018111EACF08958091E8008E77809322
:1024D000E80008958091E4009091E50045E62091A0
:1024E000EC0020FF21C02091E80020FD21C02091B8
:1024F000F001222389F0253089F02091EB0025FDA1
:102500000FC02091E4003091E5002817390739F316
:10251000415041F0C901E3CF82E0089583E008957E
:1025200081E0089584E008952091E80022FFDFCF44
:1025300080E008950E9408130E941013E0EEF0E07E
:10254000808181608083E8EDF0E080818F778083F7
:1025500019BCA7EDB0E08C918E7F8C9380818F7E2B
:1025600080831092EF0108950F931F93CF93DF9311
:102570000E9408130E941013C8EDD0E088818F7765
:10258000888388818068888388818F7D888319BC4F
:102590001092F0011092EC011092EE011092ED01F8
:1025A00000EE10E0F80180818B7F8083888181605C
:1025B000888342E060E080E00E941412E1EEF0E0E7
:1025C00080818E7F8083E2EEF0E080818160808375
:1025D000808188608083F80180818E7F80838881FC
:1025E00080618883DF91CF911F910F910895E8ED6D
:1025F000F0E080818F7E8083E7EDF0E08081816074
:10260000808384E082BF81E08093EF010C94B41258
:10261000E8EDF0E080818E7F80831092E2000895E3
:102620001092DA001092E10008951F920F920FB6F7
:102630000F9211242F933F934F935F936F937F9348
:102640008F939F93AF93BF93EF93FF938091E1009C
:1026500082FF0BC08091E20082FF07C08091E10001
:102660008B7F8093E1000E94440F8091DA0080FF0D
:102670001FC08091D80080FF1BC08091DA008E7F40
:102680008093DA008091D90080FF0DC080E189BD80
:1026900082E189BD09B400FEFDCF81E08093F001A5
:1026A0000E94150F05C019BC1092F0010E94270F5F
:1026B0008091E10080FF19C08091E20080FF15C089
:1026C0008091E2008E7F8093E2008091E200806141
:1026D0008093E2008091D80080628093D80019BC7A
:1026E00085E08093F0010E94320F8091E10084FF29
:1026F00030C08091E20084FF2CC080E189BD82E17E
:1027000089BD09B400FEFDCF8091D8008F7D8093F4
:10271000D8008091E1008F7E8093E1008091E200FB
:102720008F7E8093E2008091E20081608093E200DE
:102730008091EC01882311F084E007C08091E300D0
:1027400087FF02C083E001C081E08093F0010E9416
:10275000380F8091E10083FF29C08091E20083FF60
:1027600025C08091E100877F8093E10082E0809323
:10277000F0011092EC018091E1008E7F8093E100E6
:102780008091E2008E7F8093E2008091E200806180
:102790008093E20042E060E080E00E9414128091A9
:1027A000F00088608093F0000E942E0FFF91EF915F
:1027B000BF91AF919F918F917F916F915F914F9159
:1027C0003F912F910F900FBE0F901F9018951F9261
:1027D0000F920FB60F9211242F933F934F935F9355
:1027E0006F937F938F939F93AF93BF93CF93EF9309
:1027F000FF93C091E900CF708091EC001092E90046
:102800008091F000877F8093F00078940E942314D9
:102810001092E9008091F00088608093F000C093EE
:10282000E900FF91EF91CF91BF91AF919F918F916F
:102830007F916F915F914F913F912F910F900FBEBC
:102840000F901F9018951F93CF93DF93CDB7DEB7EE
:10285000AA970FB6F894DEBF0FBECDBFE1EFF1E04F
:102860008091F100819321E0E93FF207C9F70E94CE
:102870009D0F8091E80083FF1CC12091F1013091F0
:10288000F201832F90E08A30910508F012C1FC011B
:10289000EA5AFF4F0C94402E203881F0223809F07C
:1028A00008C18091F5018F708093E9008091EB0061
:1028B00085FB882780F91092E90006C08091ED0120
:1028C0009091EE01911182609091E800977F909332
:1028D000E8008093F1001092F100C5C0822F8D7F37
:1028E00009F0E7C0222319F0223061F0E2C08091A4
:1028F000F301813009F0DDC0333009F080E08093CE
:10290000EE0128C08091F301811124C02091F501CE
:102910002F7009F4CEC02093E9008091EB0080FF76
:1029200019C08091EB00333011F4806211C08061D6
:102930008093EB0081E090E0022E01C0880F0A94A2
:10294000EAF78093EA001092EA008091EB00886039
:102950008093EB001092E9008091E800877F86C0A9
:102960002111A7C01091F3011F778091E3008078B7
:10297000812B8093E3008091E800877F8093E800BB
:102980000E9449128091E80080FFFCCF8091E30013
:1029900080688093E300112311F083E001C082E09E
:1029A0008093F00186C02058223008F082C08091C8
:1029B000F3019091F4018C3D23E0920779F583E0D7
:1029C0008A838AE289834FB7F894DE01139620E068
:1029D0003EE051E2E32FF0E050935700E49120FFF6
:1029E00003C0E295EF703F5FEF708E2F90E0EA300A
:1029F00010F0C79601C0C0968D939D932F5F243130
:102A000049F74FBF8091E800877F8093E8006AE232
:102A100070E0CE0101960E94511114C0AE014F5FCB
:102A20005F4F6091F5010E949910009709F441C031
:102A30002091E800277F2093E800BC0189819A81DA
:102A40000E94B2118091E8008B778093E80031C03A
:102A5000203879F58091E800877F8093E8008091A5
:102A6000EC018093F1008091E8008E778093E8007C
:102A70000E9449121EC021111CC09091F301923096
:102A8000C0F48091E800877F8093E8009093EC0188
:102A90000E9449128091EC01811104C08091E300F1
:102AA00087FF02C084E001C081E08093F0010E94B2
:102AB000840F8091E80083FF0AC08091E800877F3F
:102AC0008093E8008091EB0080628093EB00AA96EF
:102AD0000FB6F894DEBF0FBECDBFDF91CF911F912F
:102AE0000895CF938091F0018823B1F08091E9009F
:102AF0008F709091EC0090FF02C090E801C090E0D0
:102B0000C92FC82B1092E9008091E80083FD0E9434
:102B10002314CF70C093E900CF910895909374016E
:102B2000809373010895E0917301F09174013097DF
:102B300021F00190F081E02D099480E00895FF924A
:102B40000F931F93CF93DF938C01E0917301F0916A
:102B50007401309799F10280F381E02D09958091FD
:102B6000D70182FF2BC080FF04C08FED96E00E944A
:102B7000FE07E80180E1F82E09ED16E08091D7010B
:102B800080FF0BC088811F928F931F930F930E9429
:102B900097080F900F900F900F90FA942196F110D4
:102BA000EDCF8091D70180FF09C087ED96E0DF91DE
:102BB000CF911F910F91FF900C94FE07DF91CF9161
:102BC0001F910F91FF900895E0917301F0917401AE
:102BD000309721F00480F581E02D0994089520912B
:102BE0007101309172018217930771F09093720115
:102BF00080937101E0917301F0917401309721F09D
:102C00000680F781E02D0994089520916F0130919D
:102C100070018217930771F09093700180936F0198
:102C2000E0917301F0917401309721F00084F185F7
:102C3000E02D0994089508950C941B160E94882293
:102C40000E941C0A0C944E23CF93C82F8091D70169
:102C500082FF1EC080FF04C088EF96E00E94FE073E
:102C60008091D70180FF0CC01F92CF9323EF36E0F5
:102C70003F932F930E9497080F900F900F900F9003
:102C80008091D70180FF04C081EF96E00E94FE078B
:102C90008C2FCF910C94D10DCF92DF92EF92FF92B7
:102CA0000F931F93CF93DF93CDB7DEB72B970FB65C
:102CB000F894DEBF0FBECDBF0E94390A36E7E32E7F
:102CC00031E0F32E00E010E0C02E802F0E94640B54
:102CD000F701D1907F01D826B1F40F5F1F4F0E305E
:102CE000110591F78FEF89838A831B820E949122BD
:102CF0008160782F9D838C8349815A816B818D817E
:102D00000E94EF1641C09091D70191FF04C08B87BC
:102D10000E946A0B8B8520E030E04D2D50E0922F11
:102D2000BA01022E02C0759567950A94E2F760FF1A
:102D300025C02E83CF82EE24E394F12C02C0EE0C4A
:102D4000FF1C9A95E2F790E08E219F2121E0892BCC
:102D500009F420E028870E9491228160782F9A87C9
:102D600089874E815F8168858A850E94EF16F80108
:102D7000EA58FE4F80818E25808306C02F5F3F4F2B
:102D80002630310561F6A9CF0E94BC26109175014D
:102D90000E9493151817A1F00E9493158093750156
:102DA0002B960FB6F894DEBF0FBECDBFDF91CF914B
:102DB0001F910F91FF90EF90DF90CF900C9424160D
:102DC0002B960FB6F894DEBF0FBECDBFDF91CF912B
:102DD0001F910F91FF90EF90DF90CF900895CF93C8
:102DE000DF93CDB7DEB72B970FB6F894DEBF0FBEDB
:102DF000CDBF4F83588769877A878B87DE0111960D
:102E000086E0FD0111928A95E9F785E0FE0137968B
:102E100001900D928A95E1F749815A816B817C81FD
:102E20008D819E810E94241E2B960FB6F894DEBFE2
:102E30000FBECDBFDF91CF910895CF93C82F8823C8
:102E400009F4C1C0823859F40E94931581FDBBC0BA
:102E500089E30E94C3200E949F2189E30CC083382C
:102E600079F40E94931580FDAEC083E50E94C320D3
:102E70000E949F2183E50E941421CF910C949F21F1
:102E8000843859F40E94931582FD9DC087E40E9406
:102E9000C3200E949F2187E4EECF8CEF8C0F813AF4
:102EA00048F48C2F0E94452B81118DC08C2F0E94DD
:102EB000C320E3CF80E28C0F883048F4C77081E0F4
:102EC00001C0880FCA95EAF70E946621D6CF8BE52C
:102ED0008C0F833078F4C53A29F0C63A31F482E891
:102EE00090E005C081E890E002C083E890E0CF91D7
:102EF0000C94EF1588E58C0F833108F064C0C83A54
:102F000039F1C93A41F1CA3A49F1CB3A51F1CC3AD7
:102F100059F1CD3A61F1C03B69F1CE3A71F1CF3A46
:102F200079F1C13B81F1C23B89F1C33B91F1C43BD3
:102F300099F1C53BA1F1C63BA9F1C73BB1F1C83B33
:102F4000B9F1C93BC1F1CA3BC9F58AE292E038C088
:102F500082EE90E035C089EE90E032C08AEE90E0DB
:102F60002FC085EB90E02CC086EB90E029C087EB6A
:102F700090E026C08CEC90E023C08DEC90E020C067
:102F800083E891E01DC08AE891E01AC082E991E0EF
:102F900017C084E991E014C081E292E011C083E29D
:102FA00092E00EC084E292E00BC085E292E008C09D
:102FB00086E292E005C087E292E002C080E090E005
:102FC000CF910C940516CF910895882309F44BC036
:102FD000823859F40E94931581FF45C089E30E940D
:102FE000C3200E949F2189E30CC0833871F40E94A2
:102FF000931580FF38C083E50E94C3200E949F2163
:1030000083E50E9414210C949F21843859F40E9476
:10301000931582FF28C087E40E94C3200E949F214D
:1030200087E4EFCF9CEF980F913A58F390E2980F16
:10303000983050F4877091E001C0990F8A95EAF7B3
:10304000892F0E946C21DFCF9BE5980F933020F4ED
:1030500080E090E00C94EF15885A833120F480E0F2
:1030600090E00C9405160895882321F00E946621B3
:103070000C949F210895882321F00E946C210C94C8
:103080009F210895CF92DF92EF92FF920F931F93AB
:10309000CF93DF93CDB7DEB728970FB6F894DEBF96
:1030A0000FBECDBF8C0185E0F801DE0111960190C5
:1030B0000D928A95E1F7F80140813181F2802581F6
:1030C00022952F7083819481892B31F03F3F31F419
:1030D00081E04F3F19F403C081E001C080E080FD32
:1030E000C6C249833A8389819A812F830E948120B5
:1030F0009E8388870E9480200E94531F4E81E42F68
:10310000E295EF70F0E0E05AFF4F2F8168850C9454
:10311000402E842F807F142F1F70882311F012956A
:10312000107FFF2059F0112309F456C2812F6887C0
:103130000E9476210E949F2168854EC2862F0E94A0
:10314000E517112309F493C2812F0E947C21289650
:103150000FB6F894DEBF0FBECDBFDF91CF911F91A8
:103160000F91FF90EF90DF90CF900C949F21342F20
:10317000307F842F8F70303211F08295807F6623EC
:1031800019F0613019F12CC0FF20B1F0222309F4AD
:1031900094C1213009F091C128960FB6F894DEBF92
:1031A0000FBECDBFDF91CF911F910F91FF90EF9098
:1031B000DF90CF900C948621222319F0213009F45E
:1031C00056C28E830E9489218E818AC1FF2021F000
:1031D000263008F04CC271C1253008F048C280C1C9
:1031E000FF2021F0222309F468C1F6C1222309F44B
:1031F00077C106C2242F26952695237030E021152D
:10320000310521F021303105C9F031C2FF2021F014
:10321000862F942F937002C080E090E028960FB61E
:10322000F894DEBF0FBECDBFDF91CF911F910F91FC
:10323000FF90EF90DF90CF900C94EF15FF2021F0DE
:10324000862F942F937002C080E090E028960FB6EE
:10325000F894DEBF0FBECDBFDF91CF911F910F91CC
:10326000FF90EF90DF90CF900C940516862FFF20F3
:1032700019F00E94422502C00E94AA2528960FB686
:10328000F894DEBF0FBECDBFDF91CF911F910F919C
:10329000FF90EF90DF90CF900C942F26842F8370B7
:1032A00009F076C0F110E3C1262F229526952770EC
:1032B000220F220F862F8F70C82ED12CE12CF12CDB
:1032C000022E04C0CC0CDD1CEE1CFF1C0A94D2F7AD
:1032D00064FF10C06FE070E080E090E004C0660F13
:1032E000771F881F991F2A95D2F760957095809552
:1032F000909503C060E070E0CB01242F26952695C1
:103300002370422F50E042305105D1F04330510537
:1033100059F16C297D298E299F294130510541F1B0
:1033200028960FB6F894DEBF0FBECDBFDF91CF91C8
:103330001F910F91FF90EF90DF90CF900C94781F2A
:103340006C297D298E299F2928960FB6F894DEBF17
:103350000FBECDBFDF91CF911F910F91FF90EF90E6
:10336000DF90CF900C94921F0E94781FC701B60186
:1033700028960FB6F894DEBF0FBECDBFDF91CF9178
:103380001F910F91FF90EF90DF90CF900C945E1FF4
:10339000FF2019F0842F817001C08695882309F4DD
:1033A00066C1262F229526952770220F220F862F81
:1033B0008F70C82ED12CE12CF12C022E04C0CC0C25
:1033C000DD1CEE1CFF1C0A94D2F764FF10C06FE0F6
:1033D00070E080E090E004C0660F771F881F991F9F
:1033E0002A95D2F7609570958095909503C060E01E
:1033F00070E0CB01242F269526952370422F50E0B4
:1034000042305105D1F04330510559F16C297D29E5
:103410008E299F294130510541F128960FB6F89425
:10342000DEBF0FBECDBFDF91CF911F910F91FF90F7
:10343000EF90DF90CF900C944C206C297D298E2941
:103440009F2928960FB6F894DEBF0FBECDBFDF913F
:10345000CF911F910F91FF90EF90DF90CF900C9440
:1034600066200E944C20C701B60128960FB6F8943A
:10347000DEBF0FBECDBFDF91CF911F910F91FF90A7
:10348000EF90DF90CF900C943220603FC9F118F498
:10349000603E50F49CC0623F09F461C008F44BC028
:1034A000633F09F470C093C0162F1F70842F8F7173
:1034B000FF2099F00E94CB1F812F28960FB6F89419
:1034C000DEBF0FBECDBFDF91CF911F910F91FF9057
:1034D000EF90DF90CF900C9434180E94EC1F812F56
:1034E00028960FB6F894DEBF0FBECDBFDF91CF9107
:1034F0001F910F91FF90EF90DF90CF900C943B18AD
:10350000FF20A9F0253008F0B2C0842F8F712896D3
:103510000FB6F894DEBF0FBECDBFDF91CF911F91E4
:103520000F91FF90EF90DF90CF900C9411202630F8
:1035300008F09DC0EACFFF20A1F0842F8F7128965C
:103540000FB6F894DEBF0FBECDBFDF91CF911F91B4
:103550000F91FF90EF90DF90CF900C94CB1FFF2046
:1035600061F3842F8F7128960FB6F894DEBF0FBEDB
:10357000CDBFDF91CF911F910F91FF90EF90DF9022
:10358000CF900C94EC1FFF2091F0842F8F71289620
:103590000FB6F894DEBF0FBECDBFDF91CF911F9164
:1035A0000F91FF90EF90DF90CF900C94B61F28966C
:1035B0000FB6F894DEBF0FBECDBFDF91CF911F9144
:1035C0000F91FF90EF90DF90CF900C94AC1FFF20F5
:1035D000A1F0222309F4B1CF862F28960FB6F894D4
:1035E000DEBF0FBECDBFDF91CF911F910F91FF9036
:1035F000EF90DF90CF900C941D17222309F4B1CFE8
:10360000862F28960FB6F894DEBF0FBECDBFDF9190
:10361000CF911F910F91FF90EF90DF90CF900C947E
:10362000E5174F70C8010E94A00828960FB6F894BD
:10363000DEBF0FBECDBFDF91CF911F910F91FF90E5
:10364000EF90DF90CF900C94D11E4F70C801289658
:103650000FB6F894DEBF0FBECDBFDF91CF911F91A3
:103660000F91FF90EF90DF90CF900C94700C289604
:103670000FB6F894DEBF0FBECDBFDF91CF911F9183
:103680000F91FF90EF90DF90CF9008950E948321DB
:103690000E9458210E949F210E945D270E942F2690
:1036A00080E090E00E94EF1580E090E00C94051619
:1036B0000E9473210C94461B0E948120292F229581
:1036C0002F7030E02C3031054CF42A3031056CF489
:1036D000225031092230310590F407C02C303105D9
:1036E00051F02F30310539F00AC0803E10F0803F94
:1036F00031F481E0089593FB882780F9089580E0F4
:103700000895CF93DF9300D000D01F92CDB7DEB7DE
:103710000F900F900F900F900F90DF91CF91089521
:10372000CF93DF9300D000D000D0CDB7DEB7269680
:103730000FB6F894DEBF0FBECDBFDF91CF910895D5
:103740001F93CF93DF93C091840116E08091850190
:10375000C81799F0D0E01C9FF0011D9FF00D1124B7
:10376000EA57FE4F40815181628173818481958146
:103770000E94901B2196C770E9CFDF91CF911F91D6
:1037800008954091B6015091B7016091B8017091D0
:10379000B9018091BA019091BB010C94901BCF9319
:1037A0008091BB0182958F7009F05FC08091B80154
:1037B000882309F45AC020918401A0918501609169
:1037C000B6017091B7018091B9019091BA0131E0D1
:1037D0006F3F09F030E0B32FC6E02A1709F445C067
:1037E000009721F07F3F21F44B2F03C041E001C03F
:1037F00040E030E040FD35C0C29FF001C39FF00DB6
:103800001124EA57FE4F418174132BC04081641389
:1038100028C04281411125C043815481481759076E
:1038200010F441505109481B590B483C5105C8F44C
:103830008091BB018F7080618093BB0186E0829F85
:10384000F001839FF00D1124E557FE4F80818F70AA
:103850008061808386EB91E00E944218CF910C94A6
:10386000A01B2F5F3F4F2770B8CFCF910895CF9205
:10387000DF92EF92FF920F931F93CF93DF93CDB719
:10388000DEB762970FB6F894DEBF0FBECDBF8C01D6
:1038900085E0F801DE011D9601900D928A95E1F711
:1038A000D8014C9111965C91119712966C911297D8
:1038B0001396ED90FC9014977091B601E091B701CA
:1038C0002091B9013091BA012115310531F0EF3F56
:1038D00031F481E07F3F19F403C081E001C080E052
:1038E000B82FB170CB2E80FD6CC1D090B801DD2017
:1038F00009F4F5C0F091BB01E216F30638F0C701F8
:10390000821B930B883C910548F09BC02095309515
:103910002E0D3F1D283C310508F093C08F2F807F6E
:1039200009F052C0E51314C0741312C0D62E6111F1
:103930000FC0FF70F061F093BB010E94C11B86EBCA
:1039400091E00E9442188091BB01F80185836CC10F
:10395000EF2831F05F3F31F481E04F3F19F403C0AD
:1039600081E001C080E080FD03C081E0862701C0C6
:1039700080E0F82FF170FF2E80FF1CC08091840141
:103980002091850136E0821709F428C190E0389F24
:10399000F001399FF00D1124EA57FE4F7181571342
:1039A00006C07081471303C07281671303C001967C
:1039B0008770E9CFD62E662309F436C18091BB010A
:1039C00081608093BB0153C0E51308C0741306C027
:1039D000611104C0D8011596FC93AEC04D875E8777
:1039E0008D859E856A8B0E945C1B6A89882329F1DC
:1039F000D62E662311F12091BB01822F82958F7004
:103A000090E002970CF460C08091B6019091B701EC
:103A100098878F831986FB86EA862C87CE010796C6
:103A200051C0E51731F14D875E878D859E856A8B84
:103A30000E945C1B6A8981112EC0C8010E94421835
:103A4000A4C08F2F807F69F77E2DF98AE88A898943
:103A50000E94811B86EB91E00E944218E6EBF1E0A8
:103A600086E0DF011D928A95E9F70E94C11BD12CE7
:103A7000DBC07413D8CF6111D6CFD8011596FC9353
:103A8000C8010E944218E6EBF1E086E0DF011D92DA
:103A90008A95E9F7C9C0D62E662379F22091BB0139
:103AA000822F82958F7090E0029774F08091B6011A
:103AB0009091B7019A8389831B82FD82EC822E83C9
:103AC000CE0101960E94421886E0F801A6EBB1E013
:103AD00001900D928A95E1F70E94CF1B6FC0E2160C
:103AE000F30628F0C701821B930B9C0104C02095AC
:103AF00030952E0D3F1D283C310508F052C0D62EC2
:103B0000662309F49ACFE5132CC074132AC0809160
:103B1000BB0180FD1DC0982F92959F70C9F0D80100
:103B200015968C9315979F3039F09F5F9295907FF3
:103B30008F70892B15968C93C8010E94421886E0DD
:103B4000F801A6EBB1E001900D928A95E1F736C03D
:103B500086E0F801A6EBB1E001900D928A95E1F7BD
:103B600063C04D875E878D859E850E945C1B882380
:103B700079F086E0F801A6EBB1E001900D928A950C
:103B8000E1F70E94CF1B0E94C11BDD24D3944CC0DF
:103B90008091BB0181608093BB01C8010E944218E3
:103BA00043C07E2DF98AE88A89890E94811BE6EB51
:103BB000F1E086E0DF011D928A95E9F70E94C11BC2
:103BC00033C0662309F439CF4D875E878D859E8586
:103BD0000E945C1B882309F430CFCBCF4D875E87D2
:103BE0008D859E850E948120292F22952F7030E09F
:103BF000223031052CF49F7041F0811106C00CC0B9
:103C0000243031052CF49F7049F4805E883020F018
:103C1000C8010E944218CF2CDC2C06C0D801159692
:103C20009C91907F91F7F8CF8D2D62960FB6F89406
:103C3000DEBF0FBECDBFDF91CF911F910F91FF90DF
:103C4000EF90DF90CF9008951F93CF93DF93CDB780
:103C5000DEB72C970FB6F894DEBF0FBECDBF4F83F3
:103C6000588769877A878B879C87CE0107960E9441
:103C7000371C8823C1F02F8138858A859B85892B45
:103C800031F03F3F11F080E003C02F3FE1F781E0CA
:103C9000811147C04F81588569857A858B859C85C0
:103CA0000E94901B3EC086E0FE013796DE01119611
:103CB00001900D928A95E1F7FF81E8854A855B8541
:103CC0004115510531F0EF3F31F481E0FF3F19F428
:103CD00003C081E001C080E080FD23C02091850108
:103CE00030E0C9010196877099276091840170E0E6
:103CF00086179707F1F1F983EA835D834C8396E099
:103D0000929FD001939FB00D1124AA57BE4FFE0180
:103D1000319601900D929A95E1F7809385010E946A
:103D2000A01B16E08091840190918501891779F19B
:103D3000189FC00111248A579E4F0E94371C882368
:103D400031F1E09184011E9FF0011124EA57FE4FEA
:103D50004081518162817381848195810E94901B91
:103D60008091840190E00196877099278093840167
:103D7000D9CF0E94581B1092850110928401E6EB66
:103D8000F1E086E0DF011D928A95E9F7CACF2C9613
:103D90000FB6F894DEBF0FBECDBFDF91CF911F915C
:103DA0000895EF92FF920F931F93CF93DF939C019F
:103DB000009709F471C0F12CEE24E394E9012196F7
:103DC000F9018491843740F4843008F056C0813082
:103DD00081F0823021F160C0853709F449C0C0F11B
:103DE0009CE7980F903708F057C08F770E94E5172F
:103DF00046C089010E5F1F4FFE01849190E2980F2B
:103E0000983050F48770FE2D01C0FF0F8A95EAF7B5
:103E10008F2F0E94762115C00E941D1714C08901A2
:103E20000E5F1F4FFE01849190E2980F983068F466
:103E30008770FE2D01C0FF0F8A95EAF78F2F0E9431
:103E40007C210E949F21E8011AC00E94E517FBCF48
:103E50002E5F3F4FFE01C491CC2341F08FE99FE0DC
:103E60000197F1F700C00000C150F6CFE90107C08B
:103E7000FE01F490E901229602C00E941D178F2DC9
:103E8000882341F0EFE9FFE03197F1F700C000002F
:103E90008150F6CF9E0192CFDF91CF911F910F916C
:103EA000FF90EF90089508956093C0017093C10151
:103EB0008093C2019093C3010C94461B0F931F93F0
:103EC0000091C0011091C1012091C2013091C30144
:103ED000062B172B282B392B0093C0011093C101FF
:103EE0002093C2013093C3011F910F910C94461B84
:103EF0000F931F930091C0011091C1012091C20145
:103F00003091C30106231723282339230093C001CE
:103F10001093C1012093C2013093C3011F910F91EF
:103F20000C94461B0F931F930091C0011091C10187
:103F30002091C2013091C30106271727282739276E
:103F40000093C0011093C1012093C2013093C301BB
:103F50001F910F910C94461B1092BC011092BD0151
:103F60001092BE011092BF010C94461B41E050E03C
:103F700060E070E004C0440F551F661F771F8A95EC
:103F8000D2F74093BC015093BD016093BE01709382
:103F9000BF010C94461B41E050E060E070E004C0BB
:103FA000440F551F661F771F8A95D2F78091BC0179
:103FB0009091BD01A091BE01B091BF01842B952BC2
:103FC000A62BB72B8093BC019093BD01A093BE019B
:103FD000B093BF010C94461B41E050E060E070E0FC
:103FE00004C0440F551F661F771F8A95D2F740956E
:103FF0005095609570958091BC019091BD01A09104
:10400000BE01B091BF0184239523A623B7238093DB
:10401000BC019093BD01A093BE01B093BF010C946D
:10402000461B41E050E060E070E004C0440F551FC3
:10403000661F771F8A95D2F78091BC019091BD01D0
:10404000A091BE01B091BF0184279527A627B7276D
:104050008093BC019093BD01A093BE01B093BF01BA
:104060000C94461B0F931F930091BC011091BD014E
:104070002091BE013091BF01062B172B282B392B25
:104080000093BC011093BD012093BE013093BF018A
:104090001F910F910C94461B0F931F930091BC012D
:1040A0001091BD012091BE013091BF01062317235D
:1040B000282339230093BC011093BD012093BE0136
:1040C0003093BF011F910F910C94461B0F931F93C8
:1040D0000091BC011091BD012091BE013091BF0142
:1040E00006271727282739270093BC011093BD0105
:1040F0002093BE013093BF011F910F910C94461B7A
:104100000895CF92DF92EF92FF920F931F93CF9378
:10411000DF93EC01C090C001D090C101E090C201DA
:10412000F090C3018091BC019091BD01A091BE01AE
:10413000B091BF01C82AD92AEA2AFB2A0FE110E070
:10414000B701A601002E04C076956795579547954F
:104150000A94D2F740FF07C0BE01802F0E94930C43
:104160008130910539F40150110950F7BE0180E00A
:104170000E94930CDF91CF911F910F91FF90EF90D0
:10418000DF90CF90089590910C01992361F1909167
:104190000D01992341F1982F9695969596959F300C
:1041A00088F4E0910E01F0910F01E90FF11D877085
:1041B00021E030E001C0220F8A95EAF78181822B4D
:1041C000818308959091D70190FF2DC01F928F9306
:1041D00089E297E09F938F930E9497080F900F902A
:1041E0000F900F90089540910E0150910F0120E023
:1041F00030E09FEFFA01E20FF31F6281681799F038
:104200009F3F19F4611101C0922F2F5F3F4F2E3055
:10421000310581F79F3F39F0FA01E90FF11D97FD54
:10422000FA9582830895089590910C01992369F17C
:1042300090910D01992349F1982F96959695969511
:104240009F3090F4E0910E01F0910F01E90FF11D04
:10425000877021E030E001C0220F8A95EAF72095AF
:1042600081812823218308959091D70190FF1FC059
:104270001F928F938BE097E09F938F930E949708F4
:104280000F900F900F900F90089540910E01509154
:104290000F0120E030E0FA01E20FF31F9281981342
:1042A00001C012822F5F3F4F2E303105A1F70895D4
:1042B00081E090E0E0910E01F0910F01E80FF91F0D
:1042C0001082019680319105A9F708959091D60149
:1042D000982B9093D601089580959091D6019823BC
:1042E0009093D60108951092D60108959091D5012A
:1042F000982B9093D501089580959091D50198239E
:104300009093D50108951092D50108958093C4012A
:1043100008951092C401089540910E0150910F012B
:1043200020E030E080E0FA01E20FF31F918191116B
:104330008F5F2F5F3F4F2F303105A9F70895E09130
:104340000E01F0910F018091D6018083E0910E0162
:10435000F0910F0180819091D501892B80839091FC
:10436000C401992361F0E0910E01F0910F01808169
:10437000892B80830E948C2181111092C40180912D
:104380000E0190910F010C949F1590933B01809327
:104390003A010895CF92DF92EF92FF920F931F930D
:1043A0006C01EE24FF24C114D104E104F10421F4D2
:1043B0006B017C0180E001C080E133272F2D1E2D91
:1043C0000D2D011511052105310519F0885F6801D2
:1043D000790197018601A4E03695279517950795F1
:1043E000AA95D1F7011511052105310519F08C5F4A
:1043F0006801790197018601F2E0369527951795B6
:104400000795FA95D1F7011511052105310519F028
:104410008E5F68017901B701A6017695679557957A
:104420004795452B462B472B09F08F5F1F910F9126
:10443000FF90EF90DF90CF9008958295982F9C7C0D
:1044400096959695837344E0849F90011124922B56
:10445000892F8A7A86959575990F892B08951F93D0
:10446000CF93DF931F92CDB7DEB799830E941D22B1
:10447000182F9981892F0E941D22212F30E0322F81
:104480002227A901482BCA010F90DF91CF911F91DC
:1044900008958091F001843009F11092D80120E450
:1044A00088E190E00FB6F894A895809360000FBE65
:1044B0002093600083B7817F846083BF83B781606E
:1044C00083BF7894889583B78E7F83BF88E10FB6CA
:1044D000F89480936000109260000FBE08950895D4
:1044E0000895CF930E946F220E94390A0E94702281
:1044F000C0E08C2F0E94640B811105C0CF5FCE30CD
:10450000C1F780E001C081E0CF9108950C94581B61
:1045100082E084BD93E095BD9AEF97BD80936E00D5
:1045200008952FB7F8948091D9019091DA01A09164
:10453000DB01B091DC012FBF0895CF92DF92EF92A3
:10454000FF920F931F932FB7F8944091D901509188
:10455000DA016091DB017091DC012FBF6A017B0100
:10456000EE24FF248C0120E030E0C016D106E206E4
:10457000F30610F441505109481B590BCA011F9111
:104580000F91FF90EF90DF90CF9008951F920F92C0
:104590000FB60F9211248F939F93AF93BF93809187
:1045A000D9019091DA01A091DB01B091DC01019673
:1045B000A11DB11D8093D9019093DA01A093DB0175
:1045C000B093DC01BF91AF919F918F910F900FBE7F
:1045D0000F901F9018950E949A12F8942FEF87EA77
:1045E00091E6215080409040E1F700C0000087E054
:1045F00090EBDC018093F9019093FA01A093FB0109
:10460000B093FC012CE088E190E00FB6F894A895F7
:10461000809360000FBE20936000FFCFEF92FF9267
:104620000F931F93CF93DF93E82EF12C8F2D0E94D1
:10463000640BC0E0D0E0082F10E098010C2E02C0FF
:10464000359527950A94E2F720FD05C02196C630DE
:10465000D10599F709C06C2F7F2D80E00E94710C65
:10466000E812F4CF81E005C0F3948EE0F812DECFBB
:1046700080E0DF91CF911F910F91FF90EF9008950F
:10468000CF93C82F8CE20E940E23882321F08C2F19
:10469000CF910C940E2380E0CF910895CF930E9488
:1046A0009B24811102C00E9481248EE497E00E9425
:1046B000FE07C5E6C15049F00E94390A8FE39CE924
:1046C0000197F1F700C00000F5CF87E497E00E9462
:1046D000FE0789E20E944023811111C18AE20E94F3
:1046E000402381110E94812485E00E944023811192
:1046F0000E94EB220E94A6248093D70187E00E94AB
:104700004023882399F18BE10E944023882351F0B4
:104710009091D70191FB882780F921E0822780FBC7
:1047200091F922C08EE00E944023882351F090919D
:10473000D70192FB882780F921E0822780FB92F93C
:1047400013C080E10E9440239091D701882341F05B
:1047500093FB882780F921E0822780FB93F904C02E
:10476000892F809580FB90F99093D7018091D70194
:104770000E94AA240E94B8248093EA0180EE0E943D
:104780004023882341F08091EA01982F909590FB77
:1047900080F98093EA0189E30E944023882359F03D
:1047A0009091EA0191FB882780F921E0822780FB24
:1047B00091F99093EA0182EE0E944023882359F0F8
:1047C0009091EA0192FB882780F921E0822780FB03
:1047D00092F99093EA0186EE0E944023882359F0D3
:1047E0009091EA0193FB882780F921E0822780FBE2
:1047F00093F99093EA0183EE0E944023882359F0B5
:104800009091EA0194FB882780F921E0822780FBC0
:1048100094F99093EA0185E30E944023882359F09C
:104820009091EA0195FB882780F921E0822780FB9F
:1048300095F99093EA0181E30E944023882359F07F
:104840009091EA0196FB882780F921E0822780FB7E
:1048500096F99093EA0181E10E944023882359F060
:104860009091EA0197FB882780F921E0822780FB5D
:1048700097F99093EA018091EA010E94BC2480910B
:10488000EA0187FB882780F980930D0187E20E9467
:104890004023C82F8EE10E9440238111C2608FE126
:1048A0000E9440238111C46080E20E944023811154
:1048B000C86081E20E9440238111C06182E20E94AF
:1048C00040238111C06283E20E9440238111C064B1
:1048D00084E20E944023882311F0C06802C0CC23E8
:1048E00029F08C2F0E94B3246C2F03C00E94AF24A8
:1048F000682F70E080E090E0CF910C94541FCF912E
:1049000008956DEE7EEF80E090E00E94762E60E0EC
:1049100082E090E00E94682E60E083E090E00E94D8
:10492000682E60E084E090E00E94682E60E085E000
:1049300090E00C94682E80E090E00E94622E21E0CE
:104940008D3E9E4F09F020E0822F089582E090E096
:104950000C945A2E682F82E090E00C94682E83E02D
:1049600090E00C945A2E682F83E090E00C94682E0F
:1049700084E090E00C945A2E682F84E090E00C9430
:10498000682E8091DF0180FF0BC06091130185E0EC
:10499000689FB001112475956795759567952AC034
:1049A00081FF09C06091130185E0689FB001112467
:1049B000759567951FC082FF07C06091130185E060
:1049C000689FB001112416C04091E0014423C9F052
:1049D00060911201461788F72091130185E0289F06
:1049E00090011124429FC001439F900D112470E05B
:1049F0000E942C2E6038710540F46115710539F064
:104A000002C065E070E0862F08958FE7089581E089
:104A100008958091DF0180FF08C06091110170E06E
:104A2000759567957595679521C081FF06C0609162
:104A3000110170E07595679519C082FF04C06091FF
:104A4000110170E010C08091E0018823C1F06091F5
:104A500010018617A0F790911101989FC0011124B1
:104A600070E00E942C2E6038710528F461157105E4
:104A700021F0862F08958FE7089581E0089561E081
:104A800070E0F4CF803F21F40E94C124819504C0DE
:104A9000813F29F40E94C1248093E3010895823F5D
:104AA00021F40E94C124819504C0833F29F40E940F
:104AB000C1248093E2010895893F19F40E940925D9
:104AC00005C08A3F31F40E94092581958093E40155
:104AD00008958B3F21F40E940925819504C08C3FE5
:104AE00029F40E9409258093E5010895843F21F46B
:104AF0008091E101816017C0853F21F48091E1013F
:104B0000826011C0863F21F48091E10184600BC076
:104B1000873F21F48091E101886005C0883F31F42E
:104B20008091E10180618093E10108958D3F21F43E
:104B30008091DF0181600BC08E3F21F48091DF0105
:104B4000826005C08F3F29F48091DF0184608093EB
:104B5000DF010895803F39F48091E30187FF6CC045
:104B60001092E30169C0813F29F48091E301181696
:104B7000BCF362C09091E201823F29F497FF5CC0D0
:104B80001092E20159C0833F19F41916CCF354C0B6
:104B9000893F41F48091E40118160CF04DC0109249
:104BA000E4014AC08A3F29F48091E40187FF44C0B0
:104BB000F6CF8B3F39F48091E50187FF3DC010921D
:104BC000E5013AC08C3F29F48091E5011816BCF349
:104BD00033C0843F21F48091E1018E7F17C0853F6F
:104BE00021F48091E1018D7F11C0863F21F48091F5
:104BF000E1018B7F0BC0873F21F48091E101877F2A
:104C000005C0883F31F48091E1018F7E8093E101FE
:104C100013C08D3F21F48091DF018E7F0BC08E3F4A
:104C200021F48091DF018D7F05C08F3F29F48091B1
:104C3000DF018B7F8093DF018091E20181110EC043
:104C40008091E30181110AC08091E401811106C0C5
:104C50008091E501811102C01092E00108958091D8
:104C6000D70183FF7EC08AE897E00E94FE0780910B
:104C7000E1011F928F9385E897E09F938F930E94A5
:104C8000970883E897E00E94FE072091E201822FB7
:104C9000992787FD90959F932F9380E897E09F93A6
:104CA0008F930E9497088EE797E00E94FE0720915D
:104CB000E301822F992787FD90959F932F938BE790
:104CC00097E09F938F930E94970889E797E00E944F
:104CD000FE072091E401822F992787FD90959F93ED
:104CE0002F9386E797E09F938F930E94970884E71E
:104CF00097E00E94FE072091E501822F992787FD0A
:104D000090959F932F9381E797E09F938F930E94B5
:104D100097088EE697E00E94FE078091E0011F92BF
:104D20008F938BE697E09F938F930E94970889E675
:104D300097E00E94FE078091DF011F928F9386E625
:104D400097E09F938F930E94970883E697E00E94D5
:104D5000FE078DB79EB74C960FB6F8949EBF0FBE58
:104D60008DBF81EE91E00E94E4150E949122909304
:104D7000DE018093DD0108951F93CF93DF9380912F
:104D8000DD019091DE010E949D224091E0014423CB
:104D900021F02091140130E006C0209115015AE065
:104DA000259F900111248217930708F482C08091F7
:104DB000E2011091E301D091E401C091E50181117C
:104DC00007C0111105C0D11103C0CC2309F471C073
:104DD0004F3F19F04F5F4093E001181624F40E94F2
:104DE000C1248093E2018091E20187FF05C00E9407
:104DF000C12481958093E201111624F40E94C124FC
:104E00008093E3018091E30187FF05C00E94C124E4
:104E100081958093E3016091E201662339F110915D
:104E2000E301112319F1772767FD7095872F972FDD
:104E30000E94312D23E333E343E35FE30E94952D8A
:104E40000E94FE2C6093E201612F772767FD709529
:104E5000872F972F0E94312D23E333E343E35FE352
:104E60000E94952D0E94FE2C6093E3011D1624F4F0
:104E70000E9409258093E4018091E40187FF05C029
:104E80000E94092581958093E4011C1624F40E9458
:104E900009258093E5018091E50187FF05C00E9407
:104EA000092581958093E501DF91CF911F910C94A5
:104EB0002F26DF91CF911F910895E1EEF1E085E07B
:104EC000DF011D928A95E9F71092E0011092DF014F
:104ED00008958DEA99E00E94FE071F9281E08F936A
:104EE0001F9285E08F938FE599E09F938F930E94A7
:104EF00097080F900F900F900F900F900F900895BC
:104F00008330E9F128F4813061F0823009F10895AD
:104F1000853009F462C008F449C0863009F474C0D1
:104F2000089520911501862F90E0820F911D8F3FEB
:104F3000910520F4620F6093150103C08FEF8093F9
:104F40001501809115011F928F9388E998E072C036
:104F500020911401862F90E0820F911D8F3F9105C3
:104F600020F4620F6093140103C08FEF809314014B
:104F7000809114011F928F9386E898E05BC0209186
:104F80001301862F90E0820F911D8F3F910520F431
:104F9000620F6093130103C08FEF80931301809120
:104FA00013011F928F9383E798E044C02091120170
:104FB000862F90E0820F911D8F3F910520F4620FA4
:104FC0006093120103C08FEF809312018091120150
:104FD0001F928F938EE598E02DC020911101862FAE
:104FE00090E0820F911D8F3F910520F4620F609336
:104FF000110103C08FEF80931101809111011F9265
:105000008F9385E498E016C020911001862F90E0E0
:10501000820F911D8F3F910520F4620F6093100164
:1050200003C08FEF80931001809110011F928F9326
:105030008AE298E09F938F930E9497080F900F90B9
:105040000F900F900895833081F128F4813059F04A
:105050008230D1F00895853009F449C0B8F1863026
:1050600009F456C0089580911501681720F4861B35
:105070008093150102C010921501809115011F92B5
:105080008F938BE198E054C080911401681720F44D
:10509000861B8093140102C01092140180911401A8
:1050A0001F928F9389E098E043C0809113016817A5
:1050B00020F4861B8093130102C01092130180918B
:1050C00013011F928F9386EF97E032C080911201F7
:1050D000681720F4861B8093120102C010921201FF
:1050E000809112011F928F9381EE97E021C08091F1
:1050F0001101681720F4861B8093110102C01092E1
:105100001101809111011F928F9388EC97E010C0DC
:1051100080911001681720F4861B8093100102C053
:1051200010921001809110011F928F938DEA97E0E9
:105130009F938F930E9497080F900F900F900F905E
:105140000895CF93C82F1F928F9322EB3AE03F939D
:105150002F930E94970861E070E080E090E004C027
:10516000660F771F881F991FCA95D2F70E94541F98
:105170000F900F900F900F90CF910C94581BCF93DE
:105180008D3109F465C0B0F58E3009F4CBC100F55E
:10519000873009F49BC1A8F4863009F06AC2809177
:1051A000D701817F8E7F8093D70187EB9AE00E94A1
:1051B000FE0789EF9EE00E94FE0781E08093E701F1
:1051C00080C1883009F44FC08B3009F47CC151C2D2
:1051D000863109F4EDC138F4803109F4B6C181316A
:1051E00009F42DC246C2893109F4CBC18B3109F4CF
:1051F00086C13FC2853309F434C248F4873209F4CA
:1052000030C208F430C2893209F42BC232C283346E
:1052100038F48A3308F029C2883309F454C129C20A
:10522000833409F41EC2883409F023C20E94581B3B
:1052300088EE9EE00E94FE079FEF23ED80E39150F1
:1052400020408040E1F700C000000E94EB2239C1FD
:1052500088E09FE00E94FE070E94B82C0E949315F0
:105260000E94D10D2EC18DEF9EE00E94FE0788ECBA
:105270009CE00E94FE070E94AF241F928F9385EC52
:105280009CE09F938F930E94970883EC9CE00E9480
:10529000FE070E94A624C82F80EB9CE00E94FE0718
:1052A0001F92CF932BEA3CE03F932F930E949708E5
:1052B00089EA9CE00E94FE078FE99CE00E94FE07BD
:1052C0008C2F81701F928F932CE93CE03F932F939A
:1052D0000E9497088AE99CE00E94FE0780E99CE012
:1052E0000E94FE07C1FB882780F91F928F932DE84B
:1052F0003CE03F932F930E9497088BE89CE00E942C
:10530000FE078FE79CE00E94FE07C2FB882780F91A
:105310001F928F932CE73CE03F932F930E949708B6
:105320008AE79CE00E94FE0781E79CE00E94FE075E
:10533000C3FBCC27C0F91F92CF938EE69CE09F93CE
:105340008F930E9497088CE69CE00E94FE070E94C3
:10535000B824C82F88E59CE00E94FE071F92CF93D7
:1053600023E53CE03F932F930E94970881E59CE062
:105370000E94FE0788E39CE00E94FE078C2F81704C
:105380001F928F9325E33CE03F932F930E94970851
:105390008DB79EB780960FB6F8949EBF0FBE8DBF97
:1053A00083E39CE00E94FE078CE19CE00E94FE07E4
:1053B000C1FB882780F91F928F9329E13CE03F933E
:1053C0002F930E94970887E19CE00E94FE0785E0EA
:1053D0009CE00E94FE07C2FB882780F91F928F93F2
:1053E00022E03CE03F932F930E94970880E09CE0EE
:1053F0000E94FE078EEE9BE00E94FE07C3FB8827FB
:1054000080F91F928F932BEE3BE03F932F930E94E6
:10541000970889EE9BE00E94FE078FED9BE00E94BB
:10542000FE07C4FB882780F91F928F932CED3BE089
:105430003F932F930E9497088AED9BE00E94FE07FE
:1054400088EC9BE00E94FE07C5FB882780F91F922D
:105450008F9325EC3BE03F932F930E94970883ECBA
:105460009BE00E94FE0787EA9BE00E94FE07C6FBC6
:10547000882780F91F928F9324EA3BE03F932F9374
:105480000E94970882EA9BE00E94FE078AE99BE05F
:105490000E94FE07C7FBCC27C0F91F92CF9387E974
:1054A0009BE09F938F930E94970885E99BE00E9461
:1054B000FE078DB79EB74C960FB6F8949EBF0FBEF1
:1054C0008DBFC1E0DBC08EED9AE058C08091D7015E
:1054D000C82FC17080FF09C08BED9EE00E94FE07BF
:1054E0008091D701817F8E7F44C08FEC9EE00E9427
:1054F000FE078091D70181608093D701E2CF809130
:10550000D70181FBCC27C0F991E0C927C0FB81F905
:105510008093D701CC2319F082EC9EE025C084EB68
:105520009EE02CC08091D70182FBCC27C0F991E08E
:10553000C927C0FB82F98093D701CC2319F085EAF3
:105540009EE012C085E99EE019C08091D70183FBDF
:10555000CC27C0F991E0C927C0FB83F98093D7011C
:10556000CC2351F089E89EE00E94FE078091D7018C
:1055700081608093D70182C08CE79EE00E94FE0785
:10558000A0CF8DE69EE00E94FE0781E49EE00E948F
:10559000FE0784E09EE00E94FE0787ED9DE00E94EA
:1055A000FE0783E99DE00E94FE0788E69DE0E6CFC6
:1055B0008AE59DE00E94FE070E9493151F928F933B
:1055C00080E49DE09F938F930E94970880910C0147
:1055D0001F928F9389E29DE09F938F930E9497087B
:1055E00080916E011F928F9386E19DE09F938F9330
:1055F0000E94970880910D011F928F9383E09DE098
:105600009F938F930E9497088091D9019091DA011E
:10561000A091DB01B091DC01BF93AF939F938F9377
:105620008FEE9CE09F938F930E9497088DB79EB753
:1056300046960FB6F8949EBF0FBE8DBF42CF0E9414
:10564000581BC0910D0181E0C827C0930D01CC23E8
:1056500029F085EE9CE00E94FE0710C08AED9CE0D8
:105660008DCF80E003C08D5101C089530E94A128D5
:1056700028CF88ED9CE00E94FE07C0E08C2FCF91E0
:10568000089580E0089580E00895CF93C82F809119
:10569000E701813081F020F0823009F44CC042C132
:1056A000A0910E01B0910F018C91813169F082328D
:1056B00009F03AC109C0A0910E01B0910F018C917F
:1056C000813111F0823249F48C2F0E94412B8111DB
:1056D0002FC08C2F0E94BF282CC08C2F0E94432BE0
:1056E000811126C0C431E1F070F4CB3081F0C031BB
:1056F000D1F40E9469278AEA9AE00E94FE0782E0BC
:105700008093E70115C0C93259F0C83361F487EBC3
:105710009AE00E94FE078EEA9AE00E94FE0708C007
:105720001092E70103C188EA9AE00E94FE07FEC0DA
:1057300081E08170FDC0C43220F5CE3108F0C0C0D8
:10574000CB3099F1C8F4C73009F0D2C08AE0809319
:10575000150194E19093140193E0909313018093C9
:10576000120188E08093110188E2809310018EE499
:1057700099E00E94FE07BFC0C33149F1C431C1F0B6
:10578000B7C0CB3409F4A9C028F4C93289F0C833B2
:1057900061F0AEC0C13509F49EC0C23509F499C0AC
:1057A000CE3409F0A5C06AE09EC00E946927A3C05C
:1057B0008091E601882319F01092E6019CC08BE5E8
:1057C00099E00E94FE0781E08093E701B1C085E384
:1057D00099E00E94FE0783E299E00E94FE07809113
:1057E00015011F928F9380E299E09F938F930E94FF
:1057F00097088EE199E00E94FE078CE099E00E94F4
:10580000FE07809114011F928F9389E099E09F9386
:105810008F930E94970887E099E00E94FE0788EF27
:1058200098E00E94FE07809113011F928F9385EFED
:1058300098E09F938F930E94970883EF98E00E94CF
:10584000FE0782EE98E00E94FE07809112011F92EF
:105850008F938FED98E09F938F930E9497088DED23
:1058600098E00E94FE0788EC98E00E94FE07809175
:1058700011011F928F9385EC98E09F938F930E9464
:10588000970883EC98E00E94FE078CEA98E00E945B
:10589000FE07809110011F928F9389EA98E09F93F1
:1058A0008F930E94970887EA98E00E94FE078DB7C1
:1058B0009EB748960FB6F8949EBF0FBE8DBF1BC013
:1058C000CE51EC2FF0E0E15DFE4F80818093E60148
:1058D00012C061E003C061E006C06AE08091E601A9
:1058E0000E94802708C08091E6010E94232803C0FF
:1058F0008CE499E013C08091E601882369F01F923F
:105900008F9386E499E09F938F930E9497080F905E
:105910000F900F900F9004C083E499E00E94FE075F
:1059200081E006C01092E70180E002C080E001CF74
:10593000CF910895E1E8F0E08081886080838081E4
:10594000816080838FB7F89493E09093890090ED05
:10595000909388008FBF0895EFE6F0E08081826029
:1059600080830895EFE6F0E080818D7F8083089545
:10597000EFE6F0E0808192E08927808308951F920E
:105980000F920FB60F9211242F933F934F935F9373
:105990006F937F938F939F93AF93BF93EF93FF93F7
:1059A0008091E8019091E90101969093E90180933B
:1059B000E801811103C082E00E94D10DE091E9016C
:1059C000E695E695F0E0E85EF04FE4918091E8011D
:1059D0008E1303C080E00E94D10DFF91EF91BF9123
:1059E000AF919F918F917F916F915F914F913F9177
:1059F0002F910F900FBE0F901F90189504D06894B0
:105A0000B1118DC0089570D088F09F5790F0B92FD4
:105A10009927B751A0F0D1F0660F771F881F991F03
:105A20001AF0BA95C9F712C0B13081F077D0B1E061
:105A3000089574C0672F782F8827B85F39F0B93F71
:105A4000CCF3869577956795B395D9F73EF4909505
:105A50008095709561957F4F8F4F9F4F0895E89483
:105A600009C097FB3EF490958095709561957F4FA6
:105A70008F4F9F4F9923A9F0F92F96E9BB27939554
:105A8000F695879577956795B795F111F8CFFAF464
:105A9000BB0F11F460FF1BC06F5F7F4F8F4F9F4F95
:105AA00016C0882311F096E911C0772321F09EE8F3
:105AB000872F762F05C0662371F096E8862F70E059
:105AC00060E02AF09A95660F771F881FDAF7880F33
:105AD0009695879597F9089557FD9058440F551F4F
:105AE00059F05F3F71F04795880F97FB991F61F060
:105AF0009F3F79F087950895121613061406551FD7
:105B0000F2CF4695F1DF08C0161617061806991F42
:105B1000F1CF86957105610508940895E894BB2737
:105B200066277727CB0197F908950BD078C069D005
:105B300028F06ED018F0952309F05AC05FC01124E8
:105B4000EECFCADFA0F3959FD1F3950F50E0551F1C
:105B5000629FF001729FBB27F00DB11D639FAA27C2
:105B6000F00DB11DAA1F649F6627B00DA11D661F11
:105B7000829F2227B00DA11D621F739FB00DA11D32
:105B8000621F839FA00D611D221F749F3327A00DEC
:105B9000611D231F849F600D211D822F762F6A2F88
:105BA00011249F5750408AF0E1F088234AF0EE0F0D
:105BB000FF1FBB1F661F771F881F91505040A9F71A
:105BC0009E3F510570F014C0AACF5F3FECF3983EA2
:105BD000DCF3869577956795B795F795E7959F5F81
:105BE000C1F7FE2B880F911D9695879597F908951B
:105BF00097F99F6780E870E060E008959FEF80EC80
:105C0000089500240A941616170618060906089522
:105C100000240A9412161306140605060895092E88
:105C20000394000C11F4882352F0BB0F40F4BF2BF7
:105C300011F460FF04C06F5F7F4F8F4F9F4F089537
:105C4000991B79E004C0991F961708F0961B881FCE
:105C50007A95C9F78095089597FB072E16F400945E
:105C600007D077FD09D00E94462E07FC05D03EF4F0
:105C7000909581959F4F0895709561957F4F0895F8
:105C8000EE0FFF1F0590F491E02D0994AA1BBB1B9A
:105C900051E107C0AA1FBB1FA617B70710F0A61B2C
:105CA000B70B881F991F5A95A9F780959095BC014D
:105CB000CD010895F999FECF92BD81BDF89A99273B
:105CC00080B50895A8E1B0E042E050E00C947D2E4C
:105CD000262FF999FECF1FBA92BD81BD20BD0FB608
:105CE000F894FA9AF99A0FBE019608950E94682EC8
:105CF000272F0C94692EDC01CB01FC01F999FECF12
:105D000006C0F2BDE1BDF89A319600B40D92415043
:0A5D10005040B8F70895F894FFCF53
:105D1A002002D20DC30EA00E6C0E390E0101C50170
:105D2A0028080A03140A3F4D36203998064B0615EF
:105D3A0006F505BC052F05480561057A059A050192
:0A5D4A000203040506070809000023
:00000001FF
